:10231E00903A0175F007ED1210A7EC75F007A425A1
:10232E0083AF82900335F0A3EFF090032DE075F0AC
:10233E0007A42401F9743A35F0FA7BFF22E075F018
:10234E0007A42401F582E4343AAF8222900326E4F6
:10235E0075F001020E14900318E475F0011210BC12
:10236E00AE02AF0122FE7B007A007908900361E491
:10237E00F0A322E024FFFFE434FFFE90032EE0FCE6
:10238E00A3E0FD22AD04EDFFEEF0A3EFF090039E6F
:10239E00740FF022900326E0FCA3E0FDC39407EC3B
:1023AE00940022E475F001120E2A85F082F583E482
:1023BE00932224FFFEE434FF90032EF0A3CEF022EE
:1023CE009003321210D3E4900330F0A3F022E49085
:1023DE000326F0A3F022AF05E4F0A3EFF0E07F00B8
:1023EE00FE22741D2DF582E43403F583229FEE64E4
:0723FE0080F8EC64809822D6
:102C3E0090038E7403F0E4A3F0FFA3F012339E7E94
:102C4E003A7F007B017A03798E12237A04F0122FD9
:102C5E0040E4F508FF74092FF8E4F60FEFB406F51B
:102C6E00E490038FF090038FE0FFC3941E5015EF96
:102C7E0012234C1223737407F0122F4090038FE02F
:102C8E0004F080E17E3A7FD37B017A0379901223A0
:092C9E007A04F0122F400230F01C
:10329D00201E103017083019081233A68003121A99
:0432AD0015D21E22F6
:10321600903AD3E493600C903A00E493640360031D
:09322600122C3EE490039EF022FC
:1032480090039E12233B78087C007D007E007F0758
:06325800120D26C21E2229
:10325E0012339E90039E12234B1223737407F012A7
:05326E002F400230F0CA
:061A1B0012325EC21E2221
:0824E700900329EFF0A3EDF0D2
:1024EF00A2AFE433900337F0C2AF900329E0FFD3DC
:1024FF009B4033EF1223C0EB1490032DF090032A6F
:10250F00122381D31223FB505812231E1223CE12F3
:10251F00257B40FB1230F090032E12235D90032D8C
:10252F00E004F002250C90032AE01223C090032C44
:10253F00E014A3F0900329122381C31223FB40213F
:10254F0012231E1223CE12257B40FB1230F0900374
:10255F002E74FFF5F0120E1490032DE014F00225E7
:0C256F0043900337E024FF92AF022FE7F7
:10257B00900332E475F0011210BCAE02AF01900370
:10258B0035E475F001120E2A85F082F583E493FD94
:10259B00122ADF900330E475F001120E14C390037E
:0B25AB0031E09407900330E094002220
:05268400900317EDF0CA
:10268900A2AFE433900328F0C2AFEF14900324F013
:10269900EB14A3F0900317E014FF900324E0D39FF9
:1026A9004003022743A312234BFE1223DC1223A269
:1026B90050190FEFAA0670010E14F5828A83E4936C
:1026C900FB1223F0EBF012235A80E2900325122328
:1026D9003B9003181210D390032412234B90031B31
:1026E900F0A3EFF01223DC12236490031B1223B131
:1026F900FD122ADF12235AC3900327E0940790039F
:1027090026E0940040E190032412233B9003181221
:1027190010D31223DC1223A250101223641223F0C7
:10272900E0FD122ADF12235A80EB1230F0900324C5
:10273900E004F0A3E004F002269D900328E024FFC2
:0527490092AF022FE732
:0729C700900343EBF0AC07A5
:1029CE00A2AFE43390034BF0C2AF9003441223E462
:1029DE00900344F0A3EFF090034412239212339E1F
:1029EE0090039E12233B9003461210D3E4900349AA
:1029FE00F0900344E0FCA3E0FFECFD900343E0FB0A
:102A0E00E490036DF0D20D12240590034AEFF0FD11
:102A1E00900346122367122ADF90034412235D901F
:102A2E000349E004F0E0C3940740C61230F090036F
:102A3E009EE004F0E0C3941E40A390034BE024FFFD
:052A4E0092AF022FE72A
:072A530090034CEBF0AC070F
:102A5A00A2AFE433900353F0C2AF90034F1223E4C2
:102A6A0090034FF0A3EFF090034F12239290039E2E
:102A7A00E0FFC3941E5053EF12234C900351F0A36E
:102A8A00EFF0E490034DF0A3F090034FE0FCA3E0D5
:102A9A00FFECFD90034CE0FB9003511223B190032D
:102AAA006DF0C20D12240590034F12235D90034D61
:102ABA0012235DC390034EE0940790034DE0940007
:102ACA0040C790039EE004F080A3900353E024FFE4
:052ADA0092AF022FE79E
:05311600900357EDF0ED
:10311B0090035874FF121037EC4D4E4F6010900314
:0E312B0057E0120D65740129F9E43AFA80E2CA
:013139002273
:1031C300E475F001120E2A85F082F5832275B7A506
:0F31D30075B7F18F828E8322EEF0A3EFF0A32267
:10322F00A2AFE433FDC2AF758F031231D0E4F0F5D6
:08323F008FAF05EF24FF92AFF1
:013247002264
:1031E200A2AFE433FCC2AF758F011231D0EDF0E42F
:0931F200F58FAF04EF24FF92AF4A
:0131FB0022B1
:102EFF009003821231DBECF0A3EDF0EB4A603190DE
:102F0F000382E0FEA3E0FFA3E0FCA3E0F5828C8345
:102F1F00E0FD1231E2EB1B70011A900384E475F0AF
:102F2F0001120E14900382E475F001120E1480CB7F
:012F3F00226F
:08339E00E4900000F0A3F0220E
:1030F000900000E0FEA3E0FF12322F900000E0FEFF
:10310000A3E0FF7C007D027B007A02122EFFE49098
:063110000000F0A3F02214
:0A2ADF00A905900371EEF0A3EFF0DB
:102AE900EE54FEFE900000E0FCA3E0FD7002EE6CE7
:102AF9006044ED4C60031230F0900371E0FEEE5437
:102B0900FEFE7F00900000F0A3EFF09003731231F6
:102B1900DB7400F0A37402F07F007E02900373124D
:102B290031C3E493FD9003751231C3EDF0EF1F70CB
:102B3900011EEF4E70E6900371E0FCA3E0FDEC543A
:0E2B490001FC74022DF58274003CF583E9F066
:012B5700225B
:102F400090035C1231DB1210D390036174FFF5F033
:102F5000120E2A45F0602090035CE475F001120E19
:102F60002AAFF0FE90035EE475F0011210BC120D62
:082F70004CFD122ADF80D22281
:1031A300900394EFF0A3EDF07F0A122D7190039436
:1031B300E0FF122D71900395E0FF122D710233B6DB
:0833A6007F02122D710233B603
:06301B00121A27EF6027E6
:103021009003967403F0A37477F0123077900396AF
:10303100E475F001120E2A85F082F583EFF0123368
:07304100BDEF70E67F0122E4
:033048007F0022E4
:1032730090039FEFF07F2F122D7190039FE0FF12B9
:053283002D710233B6BD
:103288009003A0EFF07F30122D719003A0E0FF12A1
:053298002D710233B6A8
:0233C900C11C25
:102DCE0090028EE475F001120E2A85F082F58322B0
:102DDE0090028AE0FFA3E0CF900286F0A3EFF022EC
:102DEE0090028E7402F0A374C0F022900286E475F5
:102DFE00F001120E147E027FF0900286E022E0FEB9
:102E0E00A3E0FF900286E0FCA3E0FD22EE90028A92
:052E1E00F0A3EFF0221B
:10313A0090028A122E0CB50719ECB5061590028E6C
:10314A00E0FEA3E0FFEDB50709ECB5060520C502D0
:04315A00D322C32297
:0C336800758920438E08758DE8D28E22F6
:1032B10075C101E4F5C2F5C053C17F43C18043F636
:0432C100010233686B
:102FE7007E027F90900288EEF0A3EFF090028CEEC5
:102FF700F0A3EFF0900284EEF0A3EFF07E027FC023
:10300700122E1A90028EEEF0A3EFF0EE122DE6C20A
:043017001B0232B1B5
:1030C90090028C122DD1EFF090028C122DD1EDF0DF
:1030D90090028CE0B4020FA3E0B4C00A90028C7491
:0730E90002F0A37490F02235
:0733B600C21BC2C4D2C522F4
:102D7100201B2FD21B122DCE74FFF07C027DF09010
:102D8100028EE0B50408A3E0B50503122DEE122D65
:102D9100CEE4F090028EE0B50408A3E0B50503127D
:102DA1002DEE122DCEE4F090028EE0B40208A3E0E5
:102DB100B4F003122DEE122DCEEFF090028EE0B49E
:0D2DC1000208A3E0B4F003122DEE7F012202
:10304B00900288E0FCA3E0FD900284E0B50408A3A5
:10305B00E0B505037F0022900288E0FCA3E0F58237
:0C306B008C83E0B507037F01227F002268
:10307700900288E475F001120E14900288122DD187
:10308700E0FF900288E0B4020FA3E0B4C00A900208
:08309700887402F0A37490F0AC
:01309F00220E
:061A27007FFF12304B228C
:0633BD00E4FF12304B2278
:031A18000218248D
:10182400C0E0C0F0C083C082C0D075D000C000C08A
:0718340004C005C006C00757
:10183B00E5C054FE1210DC19A70819A70A19BD0C34
:10184B0019BD0E198010198012199C14199C1619A8
:10185B00731C19731E196F24196F2619322819322C
:10186B002A19402C19402E192942192944192946A5
:10187B001929501929521929541929561929881926
:10188B00298A18CBC018D5C2189DE0189DE200001C
:10189B0019C6C2C5122DF9B5060BA3E0B507069004
:1018AB000286122DF1900286122DD1E0F5C2900224
:1018BB0086E06E7003A3E06F60030219C602192065
:1018CB00122DDED2C4D2C50219C690028E122E0C76
:1018DB00B5070EECB5060A122E1AC2C5D2C40219F0
:1018EB00C68D828C83E0B4FF030219C2122DF9B5A9
:1018FB00060BA3E0B50706900286122DF190028627
:10190B00122DD1E0F5C2900286E06E7003A3E06F5A
:10191B0060030219C6900286122DF10219C69003BC
:10192B00A1E004F00219C6E5C2602890026CE065E4
:10193B00C260208013122DDEC2C5D21CE5C260131B
:10194B0090026CE065C2600BC2C4C2C5C2C1C21DAD
:10195B000219C6ADC27FFF1230C9C2C4C2C5D2C103
:10196B00D21D8057D2C58053900286E0FFA3E0CFF3
:10197B00122E1B804690028CE0FFA3E0900284CFD6
:10198B00F0A3EFF0C2C4C2C1301C30D2C5C21C8060
:10199B002A122DDEC2C4C2C1D2C5801FC2C4C2C5A9
:1019AB00201D04C2C18014ADC2E4FF1230C9D2C1E4
:0D19BB008009122DDEC2C1C2C4D2C5C2C057
:1019C800D007D006D005D004D000D0D0D082D083A4
:0519D800D0F0D0E03268
:102CA700F9F8120E5B90033F02106A90033B121073
:102CB7006AE47FFF7EFFFDFC90033B020FF9753549
:102CC7000075360175370075380122900338E02406
:102CD70009F8E6FF22900339E0FEA3E0FFD3940052
:102CE700EE648094802290033F020FED90033B0235
:102CF7000FED900338E0FF2427F8E6223395E0FD37
:062D0700FC7810020FAA87
:10330E00D206D205D204D203D202D201122CC52289
:10331E00C206C205C204C203C202C201122CC522D9
:071A3000900338EFF0AB0555
:101A3700C2AFC200122CFC900369F0FD74392BF879
:101A4700E6F9C39DFCE49400900339F0A3CCF03091
:101A5700074A900339E0FCA3E0FDC3EC648094805F
:101A6700502B742D2FF8E670027603900338E0FFB1
:101A7700242DF816E6707B742D2FF8760174392B18
:101A8700F8E6FE74272FF8A606D2008065D3ED94FA
:101A970004EC648094804051C2078040122CDC40E3
:101AA7002E900338E0242DF8E67002760390033871
:101AB700E0FD242DF816E67039742D2DF8760174A3
:101AC700392BF8E6FC74272DF8A604D2008023C32F
:101AD700EF94FCEE6480947F500FD207900338E0B8
:101AE7002427F8A601D2008009900338E0242DF8B6
:101AF700E4F6E52645256003021D05200003021DC7
:101B070005900338E0FD2409F8E6FE74632DF5829D
:101B1700E43403F583E0FDEDFFE4FCFD90033B12A5
:101B2700106A122CDC5003021BC5EE122D03122C77
:101B3700AC122CEDC006C007900369E0FFC374FF29
:101B47009FFFE49400AB07FAE4F9F8D007D0061238
:101B57000EE6122CAC90033F120FF9C000122CD2E4
:101B6700C374FF9FFFE49400FEE4FCFDD000122C39
:101B7700A9122CD2900369E0D39F90033F400A1229
:101B87000FEDE47B407A018007120FEDE47BC0FA8A
:101B9700122CA7122CBFC000122CED7810120F9731
:101BA700D000120E40122CB2D3120F865003021C23
:101BB7005F90033B1210760000FFFF021C5F90034B
:101BC70039E0FEA3E0FFC3E49FFFE49EFE122D036E
:101BD700122CAC122CEDC007900369E0FBE4FAF974
:101BE700F8D007120EE6122CAC90033F120FF9C083
:101BF70000122CD2E4FCFDFED000122CA9122CD22C
:101C0700900369E0C39F90033F500A120FEDE47BF6
:101C1700407A018007120FEDE47BC0FA122CA7125D
:101C27002CF3C004C005C006C007122CED781012B3
:101C37000F97A804A905AA06AB07D007D006D005B9
:101C4700D004120E4D122CB2D3120F86400A900305
:101C57003B12107600000000122CF3900338E0FBD3
:101C67002463F582E43403F583EFF0122CF378084C
:101C7700120F9790033B12106A74092BF8E6FFE4E2
:101C8700FCFDFE122CBFC3120F866012122CF390BC
:101C97000338E02409F8A60712329D1228043007FA
:101CA70024122CF9FE2404FDE433FC74092FF8E612
:101CB700FFD39DEC6480F874809840028015EFC3D1
:101CC7009E50388023122CF9FE74092FF8E6FFD3B3
:101CD7009E400CE4F535F536F5377538018014EE7E
:101CE70024FCFEEFC39E5013753500753601E4F5ED
:101CF70037F53875332E7534E08003122CC5D2AF13
:011D070022B9
:0233CB00C11728
:10216900E4FFFE7D807C3F120FF9020B2A900304E5
:102179001210B3900009120FBD900005121005024C
:102189000893120FED120BD51233AEE4FF1233AEE2
:102199001233C3D2FA22856163855F61855D5FAFC2
:1021A9003D1232EC8F5D2290030B120FF9E4FFFE12
:1021B9007D807C3F02088F7FCD7ECC7DCC7C3D121B
:1021C9000FF9020893120893797F7843E4FBFA0226
:1021D9000A8DE4FFFEFD7C40900307120FF9020906
:1021E90084856062855E60855C5E853D5C229003C6
:1021F9007AE0FFA3E0FDA3E0FB22783FE4FBFAF9D4
:1022090002098412106AE4FFFE2290026CE0FF903A
:102219000379E06F22E55C540FC454F0FFF0E55CEC
:1022290054F0C4540F4F22FFEC3EA3F0A3EFF090FB
:102239000380E0FEA3E07802229003040210B39029
:102249000398E0FCA3E0FD22C286D286E50825E0DA
:10225900227841120A8D783FE4FBFAF9020893FECD
:10226900E433A3F0A3CEF0900392E0C313FEA3E0FE
:1022790022900278020FED90030F12106A90030B5F
:10228900020FEDFFE433FEF0A3EFF0D394FFEE94D9
:10229900002212106AAF03AC07E4020BA1A804A93B
:1022A90005AA06AB07221210B3900005020FBDE57F
:1022B9005D540FC454F0FFF0E55D223E90039CF09D
:1022C900A3EFF090039C22E0FEA3E0FFEE4F24FF72
:1022D9009287221228049002691210B3E94A22E473
:1022E900FBFA7980783F020B2AAD07AC06ED4C2248
:1022F90090020D020FED120FED9002F402106A9098
:102309000211020FED7FCD7ECC7DCC227BCD7ACC24
:05231900783D0208936D
:031A1500C2952255
:0333D300D295226E
:0D334E00A295E43370047F0180027F00220D
:1028A100900398EEF0A3EFF0D3943FEE6480948010
:1028B100501C122248EC120B9C7B8B7AEC798178AC
:1028C100C21209847B007A40799C78458066122285
:1028D10048D39480EC648094805019EC120B9C7B5B
:1028E1005F7A98793778C11209847B647A2F79CA23
:1028F10078448040122248D394C0EC648094805084
:1029010019EC120B9C7B787AB4790178C012098496
:102911007BD77AB279CF7843801A122248EC120B16
:102921009C7B887A4679B778BE1209847B5C7A8F62
:0829310079C0784212089322DC
:1031FC0075A4CD75F22FE4F5F3F5A5F5A675F407D6
:0A320C0075D4C075E10675E2442296
:1032D90075BC4475E88075BA1F75D108E4F5BB4320
:0332E900E60822D2
:0A338B0075A14075F809E4F5A222CF
:10332E0075DA2175DB2175DC2175DD2143E610226E
:09339500E4F5B1F5A975B283223B
:102939007592107593EC75910443E6809002051227
:1029490010760000000090020D121076437F0000FF
:10295900900257121076437F000090027C12107685
:1029690041200000900272121076439600009002F6
:10297900211210763F8000009002091210760000A3
:102989000000900211121076437F000090025B1242
:102999001076437F000090028012107641200000DB
:1029A900900276E4F0A37464F09002251210763F49
:0E29B9008000009002631210763F8000002222
:0B33800075CA8F75CBFFD2CAD2AD22F8
:1019DD00E4F5D975FF8075EF021233D3900267F0ED
:1019ED00A3F0900202F0A304F0A37480F0123395DB
:1019FD001231FC1232D912338B12332E1233801264
:051A0D002939022FE75A
:102E7400FEE43390039AF0A3CEF090039AE0C313D8
:0D2E8400FEA3E090039A13FFEEF0A3EFF021
:102E91007E00900261E0FCA3E0FD120D777C007DD5
:102EA100FF120DDE7C007DFF120D77E024FFFD9007
:092EB1000261E034FFFC120D89FE
:012EBA0022F5
:1032EC00EF131313541FFEEF5407C43354E04EFF77
:0132FC0022AF
:10318100EF4E700C1221EAAF5C122E918F74800EFB
:10319100EF64014E700812219F122E918F75122F2C
:0231A100B0225A
:102EBB001222F270191221EA90039112221EF025B0
:102ECB005C122268900392122E8A8F748022ED641A
:102EDB00014C701C12219F9003911222B8122229CF
:102EEB00F0255D12226813FF900392122E8C8F75C2
:032EFB00122FB0E3
:012EFE0022B1
:1030A0001222F2700E1221EAE55C255E122E748F58
:1030B000748012ED64014C700C12219FE55D255F58
:0830C000122E748F75122FB05F
:0130C80022E5
:0425B600AB07AA06BF
:1025BA00EB4A705C1221EA90037D12221EFFF0E5BD
:1025CA005C1313543FFEA3F0E55C5403C433335445
:1025DA00C04EF9F0E55C25E025E0FEA3F0E55C5489
:1025EA00C0FDC4131354034EF0E55C2FFFE433FE21
:1025FA00E97C002FFFEC3EFEE02F122230CEC313FF
:10260A00CE13D8F9FF900380122E8C8F7402268085
:10261A00EB64014A706012219F90037D1222B81266
:10262A002229FFF0E55D1313543FFEA3F0E55D5444
:10263A0003C4333354C04EFEF0E55D25E025E0FDCA
:10264A00A3F0E55D54C0C4131354034DFDF0EFFB32
:10265A00E55D2BFBE433FAEE7E002BFFEE3AFE7CBF
:10266A0000EF2D122230CEC313CE13D8F9FF9003F8
:09267A0080122E8C8F75122FB016
:012683002234
:102BCF001222F270311221EAE55C255EFFE433FE3A
:102BDF007A00EF2560FFEA3EFEEF2562FFEA122240
:102BEF00C412223BCEC313CE13D8F9FF90039C120D
:102BFF002E8C8F748035ED64014C702F12219FE560
:102C0F005D255FFFE433FE7C00EF2561FFEC3EFEA8
:102C1F00EF2563FFEC1222C412223BCEC313CE1357
:0E2C2F00D8F9FF90039C122E8C8F75122FB0D7
:012C3D002274
:102E230090026E12107640000000900261E4F0A35D
:102E33007402F07BFF7A3179819002691210D3E436
:102E4300F508F55CF55EF560F562F564F55DF55F33
:102E5300F561F563F565F54FF550755101F552755B
:102E63005301755401755502F5567557027558028D
:012E7300223C
:10280400E4900202F0A3F0A3E0FFC3947C5008908C
:102814000202E4F0A304F0E4900267F0A3F0EFD323
:1028240094834008900267E4F0A304F0900202123B
:1028340022D0C286D2869002671222D0122251245C
:102844004FF8E6FFB40204D2878002C287C286D260
:1028540086EFB40104D2878002C287122251244F2A
:10286400F8E67004D2878002C2871222512450F8FD
:10287400E6FFB40204D2878002C287C286D286EF02
:10288400B40104D2878002C2871222512450F8E690
:0D2894007004D2878002C287C286D28622DD
:08315E00AB07AF031BEF601A81
:103166009003861210760000445C90038674FF126A
:0A3176001037EC4D4E4F60E280F080
:01318000222C
:10115A001219DD90026C30B0057432F080037433DA
:10116A00F0122E23123216123248E5B05404F576E4
:10117A0030B10343760112330E752500752632C24B
:10118A0019D2AF43E60143F601021518D215E55B01
:10119A00700302122C14605B24FD600302122612F3
:1011AA00329D0508E508C394054003E4F508E508FF
:1011BA0014600F14601414601914601E2404702241
:1011CA0080207BFF7A2E79BB801E7BFF7A3079A044
:1011DA0080167BFF7A2579B6800E7BFF7A2B79CF32
:1011EA0080067BFF7A3179819002691210D3122826
:1011FA0004802930171AA219B3921930190AC21E8B
:10120A00121A1512329D80141233D312330E800C27
:10121A0012334EEF6006121A1B1233D3122804E45B
:10122A00F55B20160302140DC21690024B120FED45
:10123A0090024F12106A900247120FED90024B1261
:10124A00106A900243120FED90024712106A900240
:10125A003F120FED90024312220C7D7F7C439002D5
:10126A003A1221E4120BD51232EC1222A01221D129
:10127A0090023F12106A900236120FED90023A1253
:10128A00106A900232120FED90023612106A900222
:10129A002E120FED90023212106A90022A120FEDEE
:1012AA0090022E12106AAC3DE4120BA11221D190C9
:1012BA00022A12106AAC44E4120BA1C004C005C091
:1012CA0006C007AC0EE4120BA1D003D002D001D0A5
:1012DA00001221CE90027812106A900278122169C7
:1012EA00600C400A9002781210763F800000AC43EE
:1012FA00E4120BA1C004C005C006C007AC0DE4127D
:10130A000BA1D003D002D001D0001221CE900253FB
:10131A0012106A900253122169600C400A9002531B
:10132A001210763F800000AC41E4120BA1C004C049
:10133A0005C006C007AC0CE4120BA1D003D002D042
:10134A0001D0001221CE90021512106A900204E513
:10135A0045F0E4FFFE7D807C3F900215122170600B
:10136A000C400A9002151210763F800000AC42E44D
:10137A00120BA1C004C005C006C007AC0BE4120BD7
:10138A00A1D003D002D001D0001208937BBC7A749A
:10139A0079397841120A8D784012226190026E12D0
:1013AA00220C7DC07C4190026E122170600C400AB2
:1013BA0090026E12107641C0000090026E120FED7C
:1013CA00120BD5900261EEF0A3EFF0E526452560F9
:1013DA0008E5261526700215257D13E4FF121A303A
:1013EA007D147F01121A307D0D7F02121A307D0C96
:1013FA007F03121A307D0E7F04121A307D0F7F058B
:10140A00121A3012301BEF7003021196900378E023
:10141A0064317026122213702112313A50FB1215D0
:10142A002C12313A50FB1221F7A3E090032CF01250
:10143A0024E712313A50FB121535900378E06432F2
:10144A007020122213701B12313A50FB12152C1203
:10145A00313A50FB1221F712268412313A50FB120C
:10146A001535900378E0642D702A12221370251224
:10147A00313A50FB90026CE0FF12328812313A5036
:10148A00FB1221F7122A5312313A50FB90026CE0F8
:10149A00FF123273900378E0642E702A12221370BE
:1014AA002512313A50FB90026CE0FF123288123159
:1014BA003A50FB1221F71229C712313A50FB900217
:1014CA006CE0FF123273900378E0B4140AD219D296
:1014DA0017121A1512329D900378E0B415081233C8
:1014EA00D3C21912330E900378E0FFB40B02D2175D
:1014FA00201903021196EF14601A04600302119670
:10150A00900379E090039EF012324812331E12289B
:10151A0004021196900379E090039EF0121A1B02BE
:10152A00119690026CE0FF1232882290026CE0FF62
:04153A0012327322D4
:102B5800E5B05404F54E30B103434E01E54E6576B9
:102B6800600CE54E6576F566757103854E76E57100
:102B780060291571E5717023E56630E011E54E2096
:102B8800E00C90025F7401F0A37490F0D21AE5662D
:102B980030E208E54E20E203755B04301A28900203
:102BA8005F74FFF5F0120E1430B105755B01C21A9F
:102BB80090025FE07002A3E0700CC21A90026CE011
:072BC800FF7D071231A3227B
:031A12000233CECE
:0533CE00C2CFD2FF3266
:0633C300E5A120E7FB225A
:0833AE00E5A120E7FB8FA3223B
:031A2D0002153E61
:10153E00C0E0C0F0C083C082C0D075D000C000C073
:0D154E0001C002C003C004C005C006C007F4
:10155B0053917FE509253F90038A12228C40099015
:10156B00038AE4F0A374FFF01222F9900205122112
:10157B007090022150091210763F800000800712F4
:10158B001076BF800000900205120FF9C000C00159
:10159B00C002C00390038AE0FEA3E0FF1228A179EA
:1015AB00A078401221D5C004C005C006C007900228
:1015BB0021120FED90027C1221E4D003D002D00156
:1015CB00D000120A8DD003D002D001D000120893A4
:1015DB0090020512220CFDFC90022112217060106A
:1015EB00400E9002051221C090020D122170401B7B
:1015FB00E4FFFEFDFC900221122170503D90020D84
:10160B001221C0900205122170502FAF3DEFC31372
:10161B00FBEF30E004EB4480FB1222F990025712EF
:10162B00229B90020D12106A900205120FF9900284
:10163B000D12181190027C12106A9002051222FFF3
:10164B001222F99002F812106A900257120FED1243
:10165B00274E90021912220C7D7F7C4390021912A7
:10166B002170600C400A900219121076437F000023
:10167B00E4FFFEFDFC900219122170500A90021932
:10168B0012107600000000C2FA7F301233AE9002C7
:10169B001912218BE50A254090038C12228C4009EC
:1016AB0090038CE4F0A374FFF0122308900209124C
:1016BB00217090022550091210763F8000008007A0
:1016CB00121076BF800000900209120FF9C000C003
:1016DB0001C002C00390038CE0FEA3E0FF1228A11F
:1016EB00E4FBFA79A07840120A8DC004C005C0064D
:1016FB00C007900225120FED9002801221E4D00357
:10170B00D002D001D000120A8DD003D002D001D06C
:10171B000012089390020912220CFDFC9002251274
:10172B0021706015401312230E7C3D90020912218B
:10173B00C89002111221704020E4FFFEFDFC9002C4
:10174B0025122170504212230E7C3D900211122162
:10175B00C8900209122170502FAF3DEF25E0FBEF2F
:10176B0030E704EB4401FB12230890025B12229B2F
:10177B0090021112106A900209120FF990021112C5
:10178B00181190028012106A9002091222FF122384
:10179B00089002F812106A90025B120FED12274E9E
:1017AB0090021D12220C7D7F7C4390021D12217032
:1017BB00600C400A90021D121076437F0000E4FF7C
:1017CB00FEFDFC90021D122170500A90021D12109A
:1017DB007600000000C2FA7F311233AE90021D1268
:0B17EB00218B122B5875E89075BB0194
:1017F600D007D006D005D004D003D002D001D00047
:10180600D0D0D082D083D0F0D0E032120FED1208C3
:0E1816008F12335BE4FBFAF97841120A8D223F
:031A2100022F7819
:102F7800C0E0C0D075D000C000C007C2EDE5BB609E
:102F880019AFBB74382FF8A6BE75E890E5BBB4142A
:102F98000575BB00800905BB800585BE4DD216D0DE
:082FA80007D000D0D0D0E032C8
:102FB000C2FA7F321233AEAF74122191C2FA7F335C
:102FC0001233AEAF75122191C2FA7F341233AE9034
:102FD0000229E0FF122191C2FA7F351233AE90022E
:072FE0003EE0FF12219122E7
:10333E001222DC600A89828A83E4FFFE12110622C1
:1032FD001222DC600B89828A837F017E0012110607
:01330D00229D
:061D08009003041210D349
:101D0E007F9A7E997D997C3E900278122170503C8C
:101D1E00E4FBFA7980784012227A120A8D794C12FD
:101D2E002315122242900001121005120B2A900365
:101D3E00046010400E1222AFE4FBFA798012225A90
:101D4E00021E6B122179122203021E6B12227A7B63
:101D5E009A7A997999783E120B2A600250547F9A9A
:101D6E007E997D197C3F9002781221705044122288
:101D7E0042900001120FBDC004C005C006C007127C
:101D8E00230E7CBD9002781221C81222A6D007D055
:101D9E0006D005D004120B2A900304500C1222AF69
:101DAE00E4FBFAF912225A8006122179122203025A
:101DBE001E6B12227A7B9A7A997919783F120B2A26
:101DCE00600250317433FFFEFD7C3F900278122189
:101DDE0070502212217612224290000D122185128D
:101DEE002242900011122185E4FBFA7980783E128E
:101DFE000984021E6B12227A7433FBFAF9783F12B1
:101E0E000B2A600250287FCD7ECC7D4C7C3F900209
:101E1E0078122170501812217612224290000D1263
:101E2E00218574AAFBFAF9783E120984802F1222BA
:101E3E007A7BCD7ACC794C783F120B2A6002501700
:101E4E007466FFFEFD7C3F900278122170500812DE
:101E5E00217612220380061222421222B290030B26
:101E6E0012106A7FCD7ECC7D4C7C3F9002151221E4
:101E7E00E479CC12231590030712220CFD7C3F90BF
:101E8E00030712217050331221DB90030B1221E451
:101E9E0012228090030F1221C81222E8506F1221D5
:101EAE00DBC004C005C006C0071221B0D003D002AB
:101EBE00D001D000120A8D021F0F9003071221B31A
:101ECE0078401222051222A6122286120A8D1222A2
:101EDE008090030F1221C81222E85031900307128E
:101EEE0021B3E4FBFAF97840120984C004C005C09E
:101EFE0006C0071221B0D003D002D001D0001209C3
:101F0E00841222A61221B690030F12106A90025369
:101F1E001221B31221E1C004C005C006C007900310
:101F2E000F120FED9002531221E4D003D002D00114
:101F3E00D00012089390031312220C7D7F7C4390E5
:101F4E0003131221E4120BD5122242EF120D651269
:021F5E002FB0A2
:011F6000225E
:031A2400022D0D83
:102D0D00C0E0C0F0C083C082C0D075D000C000C08C
:102D1D0001C002C003C004C005C006C00730D805FD
:102D2D00C2D812333E30D905C2D91232FD30DA0B7A
:102D3D00C2DA7B017A027929121D0830DB0BC2DB66
:102D4D007B017A02793E121D08D007D006D005D03E
:102D5D0004D003D002D001D000D0D0D082D083D007
:042D6D00F0D0E03290
:101F61000000000000000000000000000000000070
:101F71000001000100010001000100010002000256
:101F81000002000200030003000300030004000438
:101F9100000500050005000600060007000700080F
:101FA100000800090009000A000A000B000B000CE0
:101FB100000D000D000E000F000F001000110011A8
:101FC1000012001300140014001500160017001869
:101FD1000019001A001A001B001C001D001E001F22
:101FE10000200021002200230024002500270028D2
:101FF1000029002A002B002C002D002F0030003179
:10200100003200340035003600380039003A003C17
:10201100003D003E004000410043004400460047AF
:102021000049004A004C004D004F0050005200543E
:10203100005500570058005A005C005E005F0061C7
:102041000063006500660068006A006C006E007045
:1020510000710073007500770079007B007D007FBF
:10206100007F00810083008500870089008B008D3F
:10207100008F009000920094009600980099009BB8
:10208100009D009F00A000A200A400A600A700A937
:1020910000AB00AC00AE00AF00B100B200B400B5BF
:1020A10000B700B800BA00BB00BD00BE00C000C14F
:1020B10000C300C400C500C700C800C900CA00CCE5
:1020C10000CD00CE00CF00D100D200D300D400D586
:1020D10000D700D800D900DA00DB00DC00DD00DE2B
:1020E10000DF00E000E100E200E300E400E500E6DB
:1020F10000E700E700E800E900EA00EB00EB00EC94
:1021010000ED00EE00EE00EF00F000F100F100F252
:1021110000F300F300F400F400F500F500F600F61A
:1021210000F700F700F800F800F900F900FA00FAEA
:1021310000FB00FB00FB00FC00FC00FC00FC00FDC0
:1021410000FD00FD00FD00FE00FE00FE00FE00FEA1
:1021510000FF00FF00FF00FF00FF00FF00FF00FF86
:0821610000FF00FF00FF00FF7A
:0C337400120FED02088F9002F0020FF91A
:06274E009002F012106A77
:102754009002F8120FF99002F012337412335BE412
:10276400FBFA7980783F120B2A600840069002F445
:10277400020FED12337A9002F81233749002FC12B5
:10278400106A12337A9002F41233749002FC120F1E
:10279400F9120A8D90030012106AE4FFFE7D7F7C1B
:1027A40043900300120FF9120984120BD5C3EE648F
:1027B4008094805003E4FEFFD3EF94FFEE64809492
:1027C4008040047E007FFFEF25E0FFEE33FE74615E
:1027D4002FF582741F3EF583E493FE740193FFFD8D
:1027E400AC06EC120B9CE4FBFA797F7843120A8D59
:0F27F4009002FC120FF912098412337A12089323
:0128030022B2
:03000000020800F3
:03000300021A03DB
:03000B00021A06D0
:03001300021A09C5
:03001B00021A0CBA
:03002300021A0FAF
:03002B00021A12A4
:03003300021A1599
:03003B00021A188E
:03004300021A1B83
:03004B00021A1E78
:03005300021A216D
:03005B00021A2462
:03006300021A2757
:03006B00021A2A4C
:03007300021A2D41
:0C080000787FE4F6D8FD75817602084789
:1032C500EFFD90036FE0FB3395E0FAC3EB9D74804F
:0432D500F86A9822D9
:0824050090036AEFF0A3EDF073
:10240D00A20D9211C2132020FDD22090036EEBF08D
:10241D00C20ED20FD2127F01C2C4C214D2C530C0B7
:10242D00FDE5C054F02480607624C0601B24E0607C
:10243D00030224CC90036EE0F5C2A20EE43342C237
:10244D00C2C5E4A3F00224CE30C149301407D2C571
:10245D00C2140224CE300F0CC20FD21090036BE0C9
:10246D00F5C2805D301011C21090036AE0F5C230E4
:10247D00114FD214D20E8049200E461232C5500E85
:10248D0090036DE0F5C290036FE004F08033D2C489
:10249D00C220802D301204D2C58026D21380221284
:1024AD0032C5500CA3E5C2F090036FE004F0D2C129
:1024BD0090036FE0B5070AC220C2C1D2C48002D218
:1024CD001330130853C0BF43C040C220C2C03020D8
:0924DD000302242B900370E0FFC0
:0124E60022D3
:10088C00020C41E86480F8E933E83360110460F04D
:10089C00ED33EC337009E8FCE9FDEAFEEBFF2204D2
:1008AC0060DED3EB9FEA9EE99DE8C2E78CF0C2F7CD
:1008BC0095F0400CE8CCF8E9CDF9EACEFAEBCFFB99
:1008CC00120C0C85D0F05804700320D5B3E80470DA
:1008DC00075002B2D5020C4B92D5EC0460F7E4CC75
:1008EC00C0E0C398F8603B94186008400DD0E0FB62
:1008FC00020C23E4FBFAC9FC8028E830E406E4C9C6
:10090C00FBE4CAFCE830E305E4C9CACBFCE85407B5
:10091C006010F8C3E913F9EA13FAEB13FBEC13FCC0
:10092C00D8F130F52FC3E49CFCEF9BFFEE9AFEED63
:10093C0099FDD0E0FBEF4E4D4C701222DB03020C04
:10094C0048EC2CFCEF33FFEE33FEED33FDED30E7DE
:10095C00EB020C23EF2BFFEE3AFEED39FDD0E0FB62
:10096C0050130BBB0003020C4BED13FDEE13FEEF0B
:08097C0013FFEC13FC020C2335
:10098400EC4D6011E8497017ED33EC3304600DE46D
:10099400FCFFFEFD22E933E8330470F8020C411237
:1009A4000C0C58046009E4CC248150062850090238
:1009B4000C4B284003020C48C0E0EB4A7044B98059
:1009C40006D0E0FB020C37EF4E701CBD8008EBFF35
:1009D400EAFEE9FD80EBE98DF0A4FEE5F0020A6D84
:1009E400E9CDF9EAFEEBFFEF89F0A4FCE5F0CE894E
:1009F400F0A42EFFE435F0CD89F0A42DFEE435F00B
:100A04008067EF4E7005BD80D780C3EF8BF0A4AC38
:100A1400F0EE8BF0A42CFCE435F0F8EF8AF0A42C73
:100A2400E5F038FCE433CB8DF0A42CFCE5F03BF886
:100A3400EE8AF0A42CFCE5F038F8E433CF89F0A476
:100A44002CFCE5F038CF3400CE89F0A42FFFE5F07C
:100A54003EFEE433C98DF0A42EFEE5F039CD8AF0D4
:100A6400A42FFFE5F03EFEE43DFD33D0E0FB50074C
:100A74000BBB000F020C4BEC2CFCEF33FFEE33FEF0
:060A8400ED33FD020C231E
:100A8A00020C4BEC5D046005E859047003020C414A
:100A9A00120C0C580460F6EC4860F2EC7004FDFE8F
:100AAA00FF22C860DB2481C85009C398600250063F
:100ABA00020C489850CAF582E9294B4A7005AB8264
:100ACA00020C3775F0007C1A7880C3EF9BEE9AED22
:100ADA0099400DC3EF9BFFEE9AFEED99FDE842F0B7
:100AEA00DC23ACF0D0E0FFD0E0FED0E0FDAB82200A
:100AFA00E7101BEB60BAEC2CFCEF33FFEE33FEED94
:100B0A0033FD020C23E803F830E705C0F075F00066
:100B1A00EF2FFFEE33FEED33FD40B830E7C280AA77
:100B2A0074F8CC6480CCC86480C8F582046043C37E
:100B3A00EB9FF5F0EA9E42F0E99D42F0E89C45F011
:100B4A0060305018E5825FFFE582F42B5582FB5036
:100B5A00210ABA001D09B90019088016E5825BFB53
:100B6A00E582F42F5582FF50090EBE00050DBD0027
:100B7A00010CC3EB9FF5F0EA9E42F0E99D42F0E8D2
:0D0B8A009C45F06007CC4820E701B3EC2249
:100B970075F020800E75F010800575F0087D007ED9
:100BA700007F003392D530D503120F78EC33401015
:100BB700EF33FFEE33FEED33FDEC33FCD5F0ED22E2
:0E0BC700E5F0247EA2D513CC92E7CDCEFF221E
:100BD500EDD2E7CD33EC3392D524814006E4FFFE18
:100BE500FDFC22FCE4CFCECDCC24E0501174FF8077
:100BF500EDC3CC13CCCD13CDCE13CECF13CF047014
:070C0500F030D5DE020F788C
:0D335B00ED33EC3360065004EC6480FC227E
:100C0C00E9D2E7C933E833F892D5EDD2E7CD33EC2E
:070C1C0033FC5002B2D522A7
:100C2300EC30E7100FBF000C0EBE00080DBD000432
:100C33000BEB6014A2D5EB13FCED92E7FD2274FFDE
:100C4300FCFDFEFF22E480F8A2D574FF13FC7D8037
:030C5300E480EF4B
:10080C0002115AE493A3F8E493A34003F68001F297
:10081C0008DFF48029E493A3F85407240CC8C333ED
:10082C00C4540F4420C8834004F456800146F6DFBC
:10083C00E4800B01020408102040809033C9E47E50
:10084C00019360BCA3FF543F30E509541FFEE493B1
:10085C00A360010ECF54C025E060A840B8E493A378
:10086C00FAE493A3F8E493A3C8C582C8CAC583CAA3
:10087C00F0A3C8C582C8CAC583CADFE9DEE780BE5B
:0133CD0000FF
:100C5600E709F608DFFA8046E709F208DFFA803E80
:100C660088828C83E709F0A3DFFA8032E309F6086D
:100C7600DFFA8078E309F208DFFA807088828C83D5
:100C8600E309F0A3DFFA806489828A83E0A3F60889
:100C9600DFFA805889828A83E0A3F208DFFA804C63
:100CA60080D280FA80C680D4806980F2803380103A
:100CB60080A680EA809A80A880DA80E280CA8033A3
:100CC60089828A83ECFAE493A3C8C582C8CCC5831B
:100CD600CCF0A3C8C582C8CCC583CCDFE9DEE780EB
:100CE6000D89828A83E493A3F608DFF9ECFAA9F06A
:100CF600EDFB2289828A83ECFAE0A3C8C582C8CCC0
:100D0600C583CCF0A3C8C582C8CCC583CCDFEADED8
:100D1600E880DB89828A83E493A3F208DFF980CC3A
:100D260088F0EF60010E4E60C388F0ED2402B40433
:100D36000050B9F582EB2402B4040050AF232345DA
:060D46008223900CA6734D
:100D4C00BB010689828A83E0225002E722BBFE02A5
:090D5C00E32289828A83E49322D8
:100D6500BB010689828A83F0225002F722BBFE016D
:020D7500F32267
:100D7700EF8DF0A4A8F0CF8CF0A428CE8DF0A42E90
:020D8700FE224A
:100D8900BC000BBE0029EF8DF084FFADF022E4CC4E
:100D9900F875F008EF2FFFEE33FEEC33FCEE9DEC17
:100DA900984005FCEE9DFE0FD5F0E9E4CEFD22ED5D
:100DB900F8F5F0EE8420D21CFEADF075F008EF2FA7
:100DC900FFED33FD4007985006D5F0F222C398FD98
:050DD9000FD5F0EA2235
:100DDE00C2D5EC30E709B2D5E4C39DFDE49CFCEE30
:100DEE0030E715B2D5E4C39FFFE49EFE120D89C312
:100DFE00E49DFDE49CFC8003120D8930D507C3E40D
:060E0E009FFFE49EFE229E
:100E1400C5F0F8A3E028F0C5F0F8E5821582700269
:060E24001583E038F02206
:100E2A00A3F8E0C5F025F0F0E5821582700215837B
:060E3A00E0C838F0E822D8
:0D0E4000EF2BFFEE3AFEED39FDEC38FC2201
:0E0E4D00C3EF9BFFEE9AFEED99FDEC98FC22A0
:100E5B00E88FF0A4CC8BF0A42CFCE98EF0A42CFC36
:100E6B008AF0EDA42CFCEA8EF0A4CDA8F08BF0A4B4
:100E7B002DCC3825F0FDE98FF0A42CCD35F0FCEB13
:100E8B008EF0A4FEA9F0EB8FF0A4CFC5F02ECD39D8
:0F0E9B00FEE43CFCEAA42DCE35F0FDE43CFC2245
:100EAA0075F008758200EF2FFFEE33FECD33CDCCFF
:100EBA0033CCC58233C5829BED9AEC99E582984082
:100ECA000CF582EE9BFEED9AFDEC99FC0FD5F0D65F
:100EDA00E4CEFBE4CDFAE4CCF9A88222B800C1B989
:100EEA000059BA002DEC8BF084CFCECDFCE5F0CBC7
:100EFA00F97818EF2FFFEE33FEED33FDEC33FCEB00
:100F0A0033FB10D703994004EB99FB0FD8E5E4F9BA
:100F1A00FA227818EF2FFFEE33FEED33FDEC33FCA7
:100F2A00C933C910D7059BE99A4007EC9BFCE99A9B
:100F3A00F90FD8E0E4C9FAE4CCFB2275F010EF2FE0
:100F4A00FFEE33FEED33FDCC33CCC833C810D707E0
:100F5A009BEC9AE899400AED9BFDEC9AFCE899F81B
:0E0F6A000FD5F0DAE4CDFBE4CCFAE4C8F922AE
:0E0F7800C3E49FFFE49EFEE49DFDE49CFC228A
:100F8600EB9FF5F0EA9E42F0E99D42F0E89C45F0C1
:010F96002238
:100F9700E8600FECC313FCED13FDEE13FEEF13FF38
:030FA700D8F1225C
:100FAA00E8600FEFC333FFEE33FEED33FDEC33FCA5
:030FBA00D8F12249
:100FBD00BB010DE58229F582E5833AF583020FED3C
:100FCD005007E92582F8021108BBFE07E92582F8D2
:100FDD00021114E58229F582E5833AF58302112089
:0C0FED00E0FCA3E0FDA3E0FEA3E0FF2277
:0C0FF900E0F8A3E0F9A3E0FAA3E0FB227B
:10100500BB010DE58229F582E5833AF583020FF9E7
:101015005007E92582F8021130BBFE07E92582F861
:1010250002113DE58229F582E5833AF58302114AED
:101035007401FF3395E0FEFDFCA3A3A3E0CF2FF0E1
:10104500E582158270021583E0CE3EF0E5821582B9
:1010550070021583E0CD3DF0E5821582700215839F
:05106500E0CC3CF0228C
:0C106A00ECF0A3EDF0A3EEF0A3EFF022F9
:10107600A8828583F0D083D08212108D12108D1233
:10108600108D12108DE473E493A3C583C5F0C58358
:10109600C8C582C8F0A3C583C5F0C583C8C582C8C4
:0110A6002227
:0C10A700A42582F582E5F03583F5832254
:0910B300E0FBA3E0FAA3E0F9223E
:1010BC00F8E0FBA3A3E0F925F0F0E58215827002BD
:0710CC001583E0FA38F02261
:0910D300EBF0A3EAF0A3E9F0221E
:1010DC00D083D082F8E4937012740193700DA3A3A3
:1010EC0093F8740193F5828883E4737402936860B7
:0610FC00EFA3A3A380DFB7
:061102008A838982E47378
:0C110800E6FC08E6FD08E6FE08E6FF2213
:0C111400E2FC08E2FD08E2FE08E2FF2217
:10112000E493FC740193FD740293FE740393FF2215
:0D113000E6FB08E6F908E6FA08E6CBF8222F
:0D113D00E2FB08E2F908E2FA08E2CBF82232
:10114A00E493F8740193F9740293FA740393FB22FB
:00000001FF
